:100000000C9476000C94EE010C9428030C943503A8
:100010000C9493000C9493000C9493000C94930014
:100020000C9493000C9493000C9493000C94930004
:100030000C9493000C9493000C9493000C949300F4
:100040000C9493000C9493000C9493000C949300E4
:100050000C94930004030904200363006F00640000
:10006000650061006E0064006C0069006600650058
:100070002E0063006F006D000C034D006F007500D3
:10008000730065001201100100000008C016E803AB
:10009000000101020001090222000101008019098A
:1000A00004000001030000000921010100012234C5
:1000B000000705810308006405010902A101090187
:1000C000A1000509190129031500250195037501F2
:1000D000810295017505810305010930093109384F
:1000E0001581257F750895038106C0C011241FBEA8
:1000F000CFE5D8E0DEBFCDBF10E0A0E6B0E0EEED8A
:10010000F7E002C005900D92A236B107D9F710E0D2
:10011000A2E6B0E001C01D92A23AB107E1F70E9449
:10012000B2030C94ED030C9400001F93162F209142
:10013000730024FF07C02091740038E82327209320
:10014000740003C02AE520937300212FDC01E5E74A
:10015000F0E08D91819321501216DCF385E790E059
:10016000612F0E94EA011C5F109373001F91089594
:100170001F93CF93DF9380918400835087FDA9C0A4
:1001800090918100209180002D3209F0A0C088302C
:1001900009F09DC0CCE0D0E0C91BD109C857DF4FA2
:1001A00083EC809368008AE580936000109262007F
:1001B0008881807621F0CE010E948F037FC09A81D2
:1001C000109271008981882331F41092720021E726
:1001D00030E082E06FC0853019F49093850067C0ED
:1001E000863009F04EC08B81813041F484E890E084
:1001F000909383008093820082E13FC0823041F47B
:1002000086E990E0909383008093820082E235C07B
:100210008330F1F4992341F484E590E090938300D6
:100220008093820084E029C0913041F488E590E019
:10023000909383008093820080E21FC09230E1F4AB
:1002400088E790E090938300809382008CE015C053
:10025000813241F488EA90E0909383008093820099
:1002600089E00BC0823241F488EB90E090938300E8
:100270008093820084E301C080E090E49093620068
:100280001DC0883069F0893019F4909387000FC041
:100290008A3049F08B3059F48BE48093740007C0A6
:1002A00027E830E002C021E730E081E003C021E729
:1002B00030E080E030938300209382009F81992377
:1002C00021F49E81981708F4892F80936100109281
:1002D00084008091600084FF4DC0809161008F3F59
:1002E00009F448C0182F893008F018E0811B80936A
:1002F00061008091680098E8892780936800112345
:1003000061F1809182009091830030916200212FF1
:10031000215036FF0EC030E0A90146595F4FFC0165
:10032000A9E6B0E064916D933196A417B507D1F7B3
:100330000CC0DC0130E0A90146595F4FE9E6F0E06E
:100340006D916193E417F507D9F72F5F3F4F280FA1
:10035000391F309383002093820089E690E0612F5B
:100360000E94EA011C5F1C3019F08FEF809361003E
:100370001093600084E193B39C7031F48150D9F7FD
:100380001092850010927F00DF91CF911F91089508
:1003900085B7826085BF8BB780648BBF8BE4809309
:1003A00074008AE5809373000895A82FB92F80E028
:1003B00090E041E050EA609530E009C02D9182273D
:1003C0009795879510F084279527305EC8F36F5F67
:1003D000A8F30895EADF8D939D930895CF93CFB747
:1003E000CF93C3959B9BE9F79B9B09C09B9B07C041
:1003F0009B9B05C09B9B03C09B9B01C0A3C0DF933D
:10040000C0918100DD27C857DF4F9B9B02C0DF9161
:10041000EBCF2F930F931F9303B32FEF03FB20F921
:100420004F933F9313B34FEF012703FB21F93BE0B9
:1004300031C04E7F012F13B3216028C0102F4D7F94
:100440002260000003B329C04B7F2460012F00000D
:1004500013B32BC013B3477F28602AC04F7E03B36A
:1004600020612CC04F7D13B320622FC04F7B03B39C
:10047000206432C0422703B349934FEF0000102796
:1004800013FB20F913B31C70C9F1297F91F20127E6
:1004900003FB21F903B3237F89F2315058F1102770
:1004A00013FB22F913B3277E79F2012703FB23F90B
:1004B0002F7C81F203B3102713FB24F92F7971F2FB
:1004C00000C013B3012703FB25F92F7359F200C0B5
:1004D00003B3102713FB26F9223040F200C013B3F8
:1004E000012703FB27F9243028F64F77206813B340
:1004F0000000F9CF10E41ABF002719C03B50319516
:10050000C31BD04010E41ABF0881033CF9F00B3440
:10051000E9F020917F001981110F1213EDCF4A816C
:10052000441F093641F10D3211F0013E29F70093C5
:1005300086003F914F911F910F912F91DF91CAB784
:10054000C6FD4FCFCF91CFBFCF9118952091860098
:10055000222379F310918400112369F534306AF174
:100560003093840020938000109181003BE0311B88
:100570003093810022C0009184000130E4F40AE548
:100580004F7049F43091600034FD19C00093600051
:10059000C8E6D0E018C03091730034FD10C000935D
:1005A0007300C4E7D0E00FC02795A8F45150A9F418
:1005B000220F0000F9CF4AE503C042ED01C0432FEE
:1005C000C4E1D0E032E014B31C60AB9A14BB05B3B5
:1005D00020E41CE05F93012756E005BB279520F43B
:1005E000515021F4220FF9CF012756E000003B5A69
:1005F00005BBD0F2279528F4515029F4220F0000B2
:10060000F9CF012756E0279505BB20F4515021F47E
:10061000220FF9CF012756E02991332305BB21F69C
:10062000037F10918500110FC651D04005BB11F01A
:1006300010937F0010E41ABF086014B3137F402F9B
:10064000437F5F9100C000C005BB14BB45BB71CFA9
:100650001F920F920FB60F9211248F9380B38F9138
:100660000F900FBE0F901F9018951F920F920FB60C
:100670000F9211240F900FBE0F901F90189587B9FD
:1006800088E28A95F1F7369A349BFECF349A84B18A
:10069000089581E08BBB85E08ABB8FE59AEE0197D8
:1006A000F1F700C0000081E00E943F0380939E00AC
:1006B00082E08BBB8AE08ABBAFE5BAEE1197F1F717
:1006C00000C0000080E00E943F038093A000909152
:1006D0009F00492F481B2091A10030919E00522F6E
:1006E000531B5093640040936500889A321769F455
:1006F000891709F490988FE799EAA3E08150904018
:10070000A040E1F700C0000001C0909A80919E00D7
:100710008093A1008091A00080939F000895FC0128
:10072000808180768032D1F48181813041F483E60A
:1007300090E0909383008093820084E0089582305B
:1007400041F487E690E0909383008093820081E0FB
:1007500008958A3029F483818093670080E00895AA
:1007600080E0089583E886B98BB7806A8BBF85B730
:10077000877F85BF85B7846085BF84B78F7B84BF43
:10078000BA98C29A11BA939A2EE088E190E00FB617
:10079000F894A89581BD0FBE21BD0E94C801A49AFE
:1007A00080E007C0A895E7EBFBE03197F1F700C0C8
:1007B00000008150B9F7A4987894A8950E94B800D9
:1007C0008091730084FFF9CF0E94490386B383E6CA
:0E07D00090E064E00E949500F0CFF894FFCF17
:0207DE005AFFC0
:00000001FF
